:100000000C9466010C9483010C9483010C94C02E13
:100010000C94D72A0C9483010C9483010C948301D3
:100020000C9483010C9483010C9483010C94042B95
:100030000C9483010C9483010C9483010C94830130
:100040000C94E82A0C9483010C94F62D0C94962EB3
:100050000C9483010C9483010C9483010C94830110
:100060000C9483010C948301084AD73B3BCE016E6C
:1000700084BCBFFDC12F3D6C74319ABD56833DDAFF
:100080003D00C77F11BED9E4BB4C3E916BAAAABE0E
:10009000000000803F05A84CCDB2D44EB93836A937
:1000A000020C50B9918688083CA6AAAA2ABE000074
:1000B00000803F000D0A4772626C20312E316820AB
:1000C0005B27242720666F722068656C705D0D0ABF
:1000D00000244E005B4F50543A005B5645523A3173
:1000E0002E31682E32303139303833303A005B549B
:1000F0004C4F3A005B4739323A0033300032380017
:100100005B4700204700204D00204600205400336C
:10011000382E005B47433A47005B484C503A242452
:1001200020242320244720244920244E2024783DC5
:1001300076616C20244E783D6C696E6520244A3DC2
:100140006C696E652024534C502024432024582091
:100150002448207E2021203F206374726C2D785D1E
:100160000D0A00414C41524D3A007C413A007C4F0F
:10017000763A007C57434F3A007C506E3A007C46FA
:100180003A007C42663A007C57506F733A007C4DCF
:10019000506F733A00536C65657000446F6F723A2C
:1001A00000436865636B00416C61726D00486F6D60
:1001B00065004A6F6700486F6C643A0052756E00C4
:1001C00049646C65000D0A005B5052423A0065724A
:1001D000726F723A00000000430000004300007A92
:1001E0004300006144000061440000FA4300C8AFCE
:1001F0004800C8AF4800A00C470000FAC30000FA4E
:10020000C3000048C30A000019010AD7233C6F123B
:10021000033B00007A440000000000000000C841D9
:100220000000FA43FA000000803F6F6B0D0A005394
:100230006C656570696E6700526573746F72696E84
:1002400067207370696E646C6500526573746F72B9
:10025000696E672064656661756C74730050676DC4
:1002600020456E6400436865636B204C696D69745A
:100270007300436865636B20446F6F720044697359
:1002800061626C656400456E61626C656400436127
:100290007574696F6E3A20556E6C6F636B656400A0
:1002A000272448277C2724582720746F20756E6CDC
:1002B0006F636B00526573657420746F20636F6E9B
:1002C00074696E7565005B4D53473A0011241FBE7B
:1002D000CFEFD8E0DEBFCDBF11E0A0E0B1E0ECE5AC
:1002E000F2E702C005900D92A430B107D9F727E0DC
:1002F000A4E0B1E001C01D92A231B207E1F70E9473
:10030000EF2E0C942C390C9400008F929F92AF9298
:10031000BF92CF92DF92EF92FF920F931F93CF93F2
:10032000DF937C016B01DC01EC91F0E0EE53F94FBF
:100330008081EF018D3229F52296818101E0912C97
:10034000F0E010E020E030E0A9015E01E0EDE80F10
:10035000EA3018F5FF5FF930E0F491101150A5E094
:10036000B0E00E9405399B01AC01220F331F441FEE
:10037000551F2E0F311D411D511D2196D5018C9108
:10038000E4CF8B3219F0219600E0D9CF22968181FB
:10039000FBCF9110F2CF1F5FF0CFEE3F29F4911009
:1003A00003C099249394E9CFFF23F9F0CA01B9015E
:1003B0000E9404364B015C0120E030E0A9010E945C
:1003C000523581112BC0002309F445C0B7FAB0940F
:1003D000B7F8B094F60180829182A282B382C25CA7
:1003E000D640C150F701C083F1E08F2FDF91CF914C
:1003F0001F910F91FF90EF90DF90CF90BF90AF9043
:100400009F908F9008952AE037ED43E25CE3C501A9
:10041000B4010E94B4374B015C011E5F1F3F9CF387
:100420001F3F59F42DEC3CEC4CEC5DE3C501B401ED
:100430000E94B4374B015C01C6CF112321F220E0AA
:1004400030E040E251E4C501B4010E94B4374B01F1
:100450005C011150F2CFD6018D929D92AD92BC926B
:100460001397BDCF2FB7F8949091CB05892B80932C
:10047000CB052FBF08952FB7F8949091CA05892B0B
:100480008093CA052FBF08959FB7F8948093C9053C
:100490009FBF08959FB7F8942091C8058095822347
:1004A0008093C8059FBF08952FB7F8949091C80511
:1004B000892B8093C8052FBF0895AF92BF92CF922A
:1004C000DF92EF92FF920F931F93CF93DF93EC0194
:1004D00007E116E05C018CE0A80EB11CC990D99030
:1004E000E990F99020E030E0A901C701B6010E942F
:1004F00074371816DCF0F801219131914191519136
:100500008F01C701B6010E94523587FD0FC0CA1581
:10051000DB0521F780E0DF91CF911F910F91FF90D4
:10052000EF90DF90CF90BF90AF90089581E0F3CF30
:100530008F929F92AF92BF92CF92DF92EF92FF92F3
:100540000F931F93CF93DF93EB0123EFE22E25E070
:10055000F22E8C016B018CE0C80ED11C699179914F
:1005600089919991F70181909190A190B1907F012B
:100570000E940636A50194010E945C35F801619342
:100580007193819391938F01CC15DD0539F7DF913C
:10059000CF911F910F91FF90EF90DF90CF90BF9080
:1005A000AF909F908F900895CF93DF93C091C60531
:1005B000D091C7052097C9F080919C0581608093F8
:1005C0009C056091B2057091B3058091B40590913E
:1005D000B5059B01AC010E94B4376A8B7B8B8C8B79
:1005E0009D8B1092C7051092C605DF91CF9108959B
:1005F00090912406492F80912506282F90FF11C045
:1006000094E080FF10C080E241FD986021FD80648D
:1006100042FD906122FD806890931502809317023D
:10062000089590E0EECF80E0EFCF8091380682FF12
:1006300013C0289A80911502809327028091230687
:100640008250990B880F81958093260280916F00CC
:10065000826080936F0008952898ECCF9091E70511
:10066000911105C0811104C02C981092F1050895D4
:10067000803119F42D982C9AF8CF2D9AFCCF249A1A
:10068000259A2C980895E091260191E09E0F9936C5
:1006900009F490E020919001291761F0F0E0E95D04
:1006A000FE4F8083909326018091C10080628093E9
:1006B000C10004C02091C80524FFECCF0895CF935A
:1006C000DF93C2ECD6E08991811103C0DF91CF9115
:1006D00008950E944303F7CF1092CC0590913806FD
:1006E00097FD03C090E29093CC05882331F0809170
:1006F000CC0590E289278093CC0508958F929F9234
:10070000AF92BF92CF92DF92EF92FF920F931F931F
:10071000CF93DF93CDB7DEB72D970FB6F894DEBF3A
:100720000FBECDBF6B017C01042F20E030E0A9019A
:100730000E94523587FF07C08DE20E944303F7FAFB
:10074000F094F7F8F094102F123008F054C000FF26
:100750000AC020E030E040E251E4C701B6010E9447
:10076000B4376B017C0120E030E040E05FE3C7017B
:10077000B6010E945D340E94CE3510E03AE0832E2F
:10078000912CA12CB12CE12FF0E0611571058105B0
:100790009105E9F581E090E08C0F9D1FE80FF91FAE
:1007A00080E3101708F445C0101309C0E1E0F0E041
:1007B000EC0FFD1FE10FF11D80E380831F5FEE242E
:1007C000E394F12CEC0EFD1EE10EF11C111134C06E
:1007D0002D960FB6F894DEBF0FBECDBFDF91CF913F
:1007E0001F910F91FF90EF90DF90CF90BF90AF904F
:1007F0009F908F90089520E030E048EC52E4C701CC
:10080000B6010E94B4376B017C0112509DCFEE24DB
:10081000E394F12CEC0EFD1EEE0EFF1EA5019401DB
:100820000E94DD38605DF7016083B901CA011F5F76
:10083000AACF1F5F8193B5CF101303C08EE20E9431
:100840004303F70182917F010E9443031150BECF01
:100850002091380640E020FF07C02BE832E441E257
:100860005DE30E94B43741E00C947E03209138068A
:1008700043E020FF07C02BE832E441E25DE30E9441
:10088000B43744E00C947E030F931F93CF938C01F5
:10089000C0E0F80161917191819191918F010E9465
:1008A0003604C23019F08CE20E944303CF5FC3309C
:1008B00081F7CF911F910F910895CF93DF938436E5
:1008C00058F06AE00E94BD38C0E3C90F6AE00E9498
:1008D000BD38D0E3D90F04C0C0E0D0E08A30B0F713
:1008E000805D0E944303DD2319F08D2F0E94430396
:1008F000CC2329F08C2FDF91CF910C944303DF910F
:10090000CF910895CF93DF93EC01FE01849121965E
:10091000811103C0DF91CF9108950E944303F5CF69
:1009200085EC91E00C948204CF93C82F8EEC91E07B
:100930000E9482048C2F0E945D04CF910C9490043D
:10094000811104C08AE292E00C9482040C94940415
:10095000CF92DF92EF92FF92CF93DF93D82F6A016D
:100960007B01C22F84E20E9443038D2F0E945D040D
:100970008DE30E9443034C2FC701B6010E947E0302
:10098000DF91CF91FF90EF90DF90CF900C94900487
:10099000CF93DF93D82FC62F84E20E9443038D2F7D
:1009A0000E945D048DE30E9443038C2F0E945D042E
:1009B000DF91CF910C949004EF92FF920F931F93CD
:1009C000CF93DF936091230670E080E00E94C8041B
:1009D0006091260670E081E00E94C80460912406C0
:1009E00070E082E00E94C8046091250670E083E018
:1009F0000E94C8046091380662FB662760F970E0C7
:100A000084E00E94C8046091380666FB662760F99E
:100A100070E085E00E94C80480913806082E000C22
:100A2000990B692F661F6627661F70E086E00E949B
:100A3000C8046091270670E08AE00E94C8044091D3
:100A400028065091290660912A0670912B0623E012
:100A50008BE00E94A80440912C0650912D066091D5
:100A60002E0670912F0623E08CE00E94A80460916E
:100A70003806617070E08DE00E94C804609138060D
:100A800065FB662760F970E084E10E94C80460910C
:100A9000380663FB662760F970E085E10E94C804B0
:100AA000609138066295617070E086E10E94C8042A
:100AB0006091390670E087E10E94C80440913A06CF
:100AC00050913B0660913C0670913D0623E088E121
:100AD0000E94A80440913E0650913F066091400656
:100AE0007091410623E089E10E94A80460914206CA
:100AF000709143068AE10E94C804409144065091D7
:100B00004506609146067091470623E08BE10E94FE
:100B1000A8044091300650913106609132067091E0
:100B2000330620E08EE10E94A804409134065091E3
:100B30003506609136067091370620E08FE10E94FD
:100B4000A80470E060E080E20E94C80484E6F82E09
:100B500010E0C3EFD5E000E0E02EEF0C123011F111
:100B6000133069F11130C9F0488159816A817B8164
:100B700023E08E2D0E94A8040F5F2496033061F7B6
:100B80008AE0F80E1F5F8CE8F812E3CFDF91CF9177
:100B90001F910F91FF90EF9008954C855D856E85B4
:100BA0007F85E6CF20E030E041E655E4688D798D21
:100BB0008A8D9B8D0E945C35AB01BC01D9CF4CA1C5
:100BC0005DA16EA17FA17058D3CF8DE50E94430334
:100BD0000C949004CF93DF93CDB7DEB72C970FB66C
:100BE000F894DEBF0FBECDBF88EC91E00E94820476
:100BF00069ED75E0CE0101960E949802CE01019642
:100C00000E9444048AE30E9443038091EB050E9402
:100C10005D040E94E5052C960FB6F894DEBF0FBE6A
:100C2000CDBFDF91CF910895EAE0F1E0ADECB5E002
:100C30004D915D916D917C911397408351836283B7
:100C4000738314964D915D916D917C9117974483B8
:100C500055836683778318968D919D910D90BC91F5
:100C6000A02D80879187A287B3870895BF92CF92E6
:100C7000DF92EF92FF920F931F93CF93DF937C014C
:100C8000FC0102A513A5D4A5C5A5818980FF33C0A9
:100C90006091EE0570E090E080E00E9406362AE068
:100CA00037ED43E25CE30E94B4379B01AC01B8012D
:100CB0008D2F9C2F0E94B4378B01D82FC92F20E095
:100CC00030E040E85FE3B8018D2F9C2F0E9474371D
:100CD000181624F000E010E0D0E8CFE3B8018D2F23
:100CE0009C2FDF91CF911F910F91FF90EF90DF909C
:100CF000CF90BF90089582FD17C06091ED0570E020
:100D000090E080E00E9406362AE037ED43E25CE3A3
:100D10000E94B4379B01AC01B8018D2F9C2F0E941B
:100D2000B4378B01D82FC92FF701B6A0C7A0D0A424
:100D3000F1A498014D2F5C2F6B2D7C2D8D2D9F2DB7
:100D40000E94523587FFBBCF0B2D1C2DDD2DCF2DE3
:100D5000B6CF80913D0290911E05981739F02EE292
:100D6000829FC0011124825C9D4F089590E080E035
:100D700008950E94A906892B19F082E00C94540270
:100D800008952F923F924F925F926F927F928F922F
:100D90009F92AF92BF92CF92DF92EF92FF920F930A
:100DA0001F93CF93DF9300D000D0CDB7DEB7009173
:100DB0001E05002309F486C0098339813150398327
:100DC00010913C02131709F466C0C32ED12CEEE239
:100DD0003E9FC00111249C01225C3D4F7901F90125
:100DE00076888788908CA18C628D738D848D958D8B
:100DF0009B01AC010E945D34F701268D378D40A127
:100E000051A10E94B437B62EE72EF82E9B83262FD1
:100E1000372F482F592F672D782D892D9A2D0E9415
:100E2000523587FF03C0B72C7401AB828EE28C9DD4
:100E3000F0018D9DF00D1124E25CFD4F8B2D9E2D58
:100E4000AF2DBB81828B938BA48BB58BF9818F2FB8
:100E5000F11101C080E1FF24FA94F80E30903D02B8
:100E60001F1133C0131102C00E94D402EEE21E9F74
:100E7000C0011124825C9D4F9A838983332433946B
:100E8000310EF0E13F1201C0312C8EE2282E031109
:100E900085C010933C020F900F900F900F90DF9140
:100EA000CF911F910F91FF90EF90DF90CF90BF9067
:100EB000AF909F908F907F906F905F904F903F90FA
:100EC0002F90089520E1298378CF29818EE2289FF1
:100ED00090011124225C3D4F3C832B832EE2E22EB5
:100EE0008F2C912CFE9CC0011124FC01E25CFD4F73
:100EF000FA83E983F11002C090E1F92EFA94F3101D
:100F000002C00E94D402E89CC001E99C900D11240B
:100F10009C01225C3D4F6901F90146885788608C2D
:100F2000718CA301920162897389848995890E94D9
:100F30005235882339F1F601628D738D848D958D3C
:100F40009B01AC010E945D34F601268D378D40A1D6
:100F500051A10E94B437EB81FC81228933894489F5
:100F600055890E945D344B015C01AC019B01C301BA
:100F7000B2010E947437F60118165CF4828A938AD3
:100F8000A48AB58A29813A813C832B831F11A8CF7B
:100F90006DCF428A538A648A758AF4CFC32CD12CD0
:100FA000329CC00111249C01225C3D4F7901E981F2
:100FB000FA814288538864887588F9018288938809
:100FC000A488B588A5019401C301B2010E945235DD
:100FD00087FF26C0E981FA81628D738D848D958D9E
:100FE0009B01AC010E945D34E981FA81268D378D29
:100FF00040A151A10E94B437A30192010E945D3427
:101000002B013C01AC019B01C501B4010E94743766
:10101000181634F4F701428A538A648A758A132DAC
:101020002C9CF0012D9CF00D1124E25CFD4F2689D3
:101030003789408D518D62897389848995890E9491
:101040005235811101C0132D3394F0E13F1201C0DC
:10105000312CFA82E9821BCF6F927F928F929F92FE
:10106000AF92BF92CF92DF92EF92FF920F931F93B6
:10107000CF93DF93EB018C015B018CE0A80EB11CD8
:1010800089E9682E96E7792E26E9822E3EE7932E8F
:10109000C990D990E990F99020E030E0A901C7010A
:1010A000B6010E9452358823B9F0A7019601F801D4
:1010B00060817181828193810E945C356B017C012A
:1010C000E894F7F89301A401C701B6010E947437B0
:1010D000181614F0360147010C5F1F4FCA15DB05C7
:1010E000B9F6B301C401DF91CF911F910F91FF9029
:1010F000EF90DF90CF90BF90AF909F908F907F90B8
:101100006F90089593B18091380686FF0BC09E7052
:1011100059F091FB882780F992FD8260987029F040
:10112000846008959095F3CF80E00895EBE6F0E0B9
:101130008081817F8083E8E6F0E080818E7F8083FC
:10114000089584B1817F84B985B18E6085B980911D
:10115000380683FF0BC080916B008E6080936B001C
:101160008091680081608093680008950C949608CF
:101170006DEC75E080E696E00C949802F894F9998D
:10118000FECF92BD81BD81E08FBB20B5862F822727
:10119000082E000C990B50E086239523892B49F0EB
:1011A00084E16F3F11F060BD84E08FBBF99A7894C1
:1011B00008952617E1F360BD84E2F7CF9F92AF92C6
:1011C000BF92CF92DF92EF92FF920F931F93CF9334
:1011D000DF935C018A017B01E40EF51EEB01912C8B
:1011E0006C01C61AD70ACE018C0D9D1D21E091100D
:1011F00007C0292D990C330B232F221F2227221FD2
:101200006991962E920E0E94BE08CE15DF0559F701
:10121000692DC501800F911FDF91CF911F910F9113
:10122000FF90EF90DF90CF90BF90AF909F900C9485
:10123000BE086AE090E080E00E94BE0845E550E00C
:1012400063EF75E081E090E00C94DE08F999FECF41
:1012500092BD81BD81E08FBB80B508959F92AF9212
:10126000BF92CF92DF92EF92FF920F931F93CF9393
:10127000DF935B018A017C01E40EF51EEC01912CE9
:101280006B01C81AD90AC6018C0F9D1F0E9426093E
:1012900021E0911007C0292D990C330B232F221F19
:1012A0002227221F982E920E8993CE15DF0559F71B
:1012B000C501800F911F0E94260921E030E08915A9
:1012C00011F030E020E0C901DF91CF911F910F9123
:1012D000FF90EF90DF90CF90BF90AF909F900895D8
:1012E0009091E705911105C086FF04C0439A1092C2
:1012F000F10508954398FBCFEAE0F1E08CE1DF01CE
:101300001D928A95E9F710923D0210921E0581E028
:101310008093090110923C0208954F925F926F9260
:101320007F92AF92BF92CF92DF92EF92FF920F9394
:101330001F93CF93DF93EC015C012CE0A20EB11C54
:101340008C01C12CD12C7601F80141905190619013
:1013500071908F0120E030E0A901C301B2010E9429
:101360005235882371F0A3019201C301B2010E949A
:10137000B4379B01AC01C701B6010E945D346B011B
:101380007C010A151B0501F7C701B6010E945338FD
:101390006B017C01AC019B0160E070E080E89FE3A1
:1013A0000E945C352B013C01699179918991999159
:1013B0005E01F4E0AF1AB108A30192010E94B437B4
:1013C000F5016083718382839383C017D10761F72E
:1013D000C701B601DF91CF911F910F91FF90EF9060
:1013E000DF90CF90BF90AF907F906F905F904F90C5
:1013F00008952F923F924F925F926F927F928F92B9
:101400009F92AF92BF92CF92DF92EF92FF920F9393
:101410001F93CF93DF93CDB7DEB7C654D1090FB674
:10142000F894DEBF0FBECDBF2091EA052AA320FDB0
:10143000E1C624702BAB30911E0539AF4EE2349FCC
:10144000C0011124DC01A25CBD4F2396BFAFAEAF3B
:101450002397BAA1B270BCAB40913D024AAF4F5F37
:101460004D8F403109F458C74BAF5EE2ABAD5A9F88
:10147000C0011124FC01E05BFD4F2596FFAFEEAFEC
:10148000259790911F0580912005981709F4B2C601
:101490008091C6059091C705892B09F079C0EBA909
:1014A000EE2309F40FC223962EAD3FAD2397309360
:1014B000C7052093C6054091C6055091C7055A87B8
:1014C0004987452B09F496C610919C0510FF01C26F
:1014D00010929C051092AE051092AF051092B005C7
:1014E0001092B105A985BA855A962D913D914D91DD
:1014F0005C915D9729833A834B835C8360E070E065
:1015000080E09FE30E945C356D837E838F839887A4
:10151000E985FA85468C578C60A071A082889388F3
:10152000A488B588FCA9FF2309F4A1C222E0209376
:10153000AD05A50194010E94B4379B01AC01C30124
:10154000B2010E945C346B017C0120E030E0A90113
:101550000E94523587FF7AC229813A814B815C8192
:10156000CA01B9010E945D34A30192010E94B437FF
:101570009B01AC01C501B4010E945C340E94533848
:101580006093BA057093BB058093BC059093BD052D
:1015900080914505482F50E05A8B498B86E0849F07
:1015A000F001859FF00D1124EF5DFA4F80919B05AE
:1015B0008483A091C605B091C705BE87AD875E96AE
:1015C000BC91BFA3ED85FE85F78DF8A7AD85BE85DF
:1015D0009096BC91B9A7ED85FE85F1A1FAA720915F
:1015E000A9053091AA054091AB055091AC056FA1BA
:1015F00078A58B2F9F2F0E945C346DAB7EAB8FAB99
:1016000098AF20E030E0A9010E94523587FF04C066
:101610001DAA1EAA1FAA18AE2091B6052D8B3091C7
:10162000B7053E8B4091B8054F8B5091B905588F47
:101630008091BE058E8F9091BF059F8FA091C005B0
:10164000A8A3B091C105B9A3E091C205EBA7F091A1
:10165000C305FCA72091C4052DA73091C5053EA761
:101660003090B2052090B3054091B40527964FAF56
:1016700027975091B50526965FAF26978091AD05C7
:1016800089879091AE059FA7A091AF05A8ABB091B7
:10169000B005B9ABE091B105EAABF091BA05FDAF89
:1016A0002091BB052EAF3091BC053FAF4091BD05E9
:1016B00021964FAF21972BA53CA54DA55EA56E8D1C
:1016C0007F8D88A199A10E945235811159C352E0A2
:1016D0005CAF9FA1998FA8A5AA8FB9A5BB8FEAA5DA
:1016E000EC8F8EE3C82E83ECD82E8EE2E82E89E3B1
:1016F000F82E412C512C3201A70196012BA33CA3BB
:101700004DA35EA35985513009F4F7C3AD85BE855D
:10171000513008F46FC3533009F025C45A962D9107
:101720003D914D915C915D97C701B6010E94B43720
:101730004B015C012D893E894F89588D632D722D97
:1017400027968FAD279726969FAD26970E945C34EB
:101750009B01AC01C501B4010E94743787FD1AC317
:101760002E8D3F8D48A159A16FA178A589A59AA575
:101770000E945C349B01AC010E945D346B017C01D2
:101780002D893E894F89588D632D722D27968FADF7
:10179000279726969FAD26970E945D349B01AC014A
:1017A000C701B6010E945C356B017C013D882E8823
:1017B000BF892796BFAF2797E88D2696EFAF26976C
:1017C0000E8D1F8DF8A1F98329A12D8331E0398772
:1017D000A7019601C301B2010E945D342B013C01B7
:1017E0002BA13CA14DA15EA10E94523587FF3CC4B4
:1017F000A30192016BA17CA18DA19EA10E945C34EA
:101800006B017C01980149815D816FA578A989A947
:101810009AA90E94523587FDB6C2832D922D279634
:10182000AFAD27972696BFAD26978093B2059093CC
:10183000B305A093B405B093B50539853093AD05D4
:101840002091A5053091A6054091A7055091A805C6
:10185000B80189819D810E94B43769877A878B8717
:101860009C870E943B356B017C016091A1057091C2
:10187000A2058091A3059091A4050E943B354B01E0
:101880005C01A70196010E945C340E94D5356D87EA
:101890007E878F87988BA6E089899A89A89FF00117
:1018A000A99FF00D1124EF5DFA4F2D853E85318300
:1018B0002083232B09F008C45CA9552309F404C430
:1018C0008AA195C40E94A9069093C7058093C60576
:1018D000F2CD80919B058F5F853009F480E0809385
:1018E0009B05482F50E091E1949FF001959FF00DEA
:1018F0001124EA5BFA4FA985BA8550969C915097BE
:10190000908BE1E18E9FC001112430E020E0CD906A
:10191000DD90ED90FD90FC01E20FF31FEA5BFA4FC2
:1019200063E0CC0CDD1CEE1CFF1C6A95D1F7C08275
:10193000D182E282F3822C5F3F4F2C30310539F7A0
:10194000A985BA851C966D917D918D919C911F976B
:10195000B1E1B49F9001B59F300D1124F901EA5B0C
:10196000FA4F6B017C0123E0CC0CDD1CEE1CFF1C4C
:101970002A95D1F7C486D586E686F7860E94043676
:101980006093A1057093A2058093A3059093A4058D
:10199000E985FA85268D378D40A151A10E945C35DD
:1019A0009B01AC012093A5053093A6054093A705A4
:1019B0005093A80560E070E080EA9FE30E945C35E8
:1019C0006093A9057093AA058093AB059093AC052D
:1019D00010929D0510929E0510929F051092A005F1
:1019E000FCA9F11102C013FF20C06091BA057091EB
:1019F000BB058091BC059091BD056093B2057093C5
:101A0000B3058093B4059093B5059B01AC010E948A
:101A1000B437A985BA8552966D937D938D939C9327
:101A20005597177F10939C0555CDE985FA856289F6
:101A30007389848995890E9453386093B2057093A5
:101A4000B3058093B4059093B50544CDC092AE051F
:101A5000D092AF05E092B005F092B1051092BA05B0
:101A60001092BB051092BC051092BD0591CD10924D
:101A7000AD054092BE055092BF056092C0057092C0
:101A8000C1053BA9332309F46AC01092BA0510922C
:101A9000BB051092BC051092BD05C12CD12C76015E
:101AA00089859A850E9436066D877E878F87988BF9
:101AB0009B01AC010E94B43769877A878B879C872A
:101AC000A50194010E94523587FF8BC029853A8574
:101AD0004B855C85C501B4010E945C342D813E813B
:101AE0004F8158850E94B4379B01AC01C301B201FC
:101AF0000E945C346093BE057093BF058093C0055F
:101B00009093C10520E030E0A9010E9452351816DB
:101B10000CF441C0B2E0B093AD0529813A814B810C
:101B20005C81CA01B9010E945D34A30192010E9447
:101B3000B4379B01AC01C501B4010E945C340E9422
:101B400053386093BA057093BB058093BC0590939E
:101B5000BD0580919C05886080939C0519CD49AD99
:101B60005BADC12CD12C7601451741F02596AEAD69
:101B7000BFAD2597CD90DD90ED90FC90C701B601EB
:101B80000E9453386093BA057093BB058093BC05DF
:101B90009093BD0585CFA701960169857A858B85D0
:101BA0009C850E945C342D813E814F8158850E9426
:101BB000B4376093C2057093C3058093C4059093B6
:101BC000C5052D853E854F8558892093B6053093F0
:101BD000B7054093B8055093B90533E03093AD0590
:101BE000D7CCA7019601C501B4010E945C342D81B8
:101BF0003E814F8158850E94B437A30192010E9413
:101C00005D3420E030E040E05FE30E94B437698B50
:101C10007A8B8B8B9C8B20E030E0A9010E9474377B
:101C200018160CF094C0A301920169897A898B89F6
:101C30009C890E94523587FF88C0A701960169855B
:101C40007A858B859C850E945C342D813E814F81F5
:101C500058850E94B4379B01AC012093C205309394
:101C6000C3054093C4055093C50569897A898B895A
:101C70009C890E9474371816BCF58D859E85AF85AA
:101C8000B8898093B6059093B705A093B805B09333
:101C9000B905A501940169857A858B859C850E948B
:101CA0005235811104C091E09093AD0571CCA5012E
:101CB000940169857A858B859C850E945C342D8191
:101CC0003E814F8158850E94B4379B01AC01C3010E
:101CD000B2010E945C346093BE057093BF0580938F
:101CE000C0059093C10554CC29893A894B895C89F8
:101CF0002093BE053093BF054093C0055093C105A6
:101D00002093C2053093C3054093C4055093C50585
:101D100029813A814B815C81CA01B9010E945D34FD
:101D200029893A894B895C890E94B437A7019601B9
:101D30000E945D340E9453386093B6057093B705D6
:101D40008093B8059093B90523CC32E047CF8091BA
:101D5000BA059091BB05A091BC05B091BD0510924C
:101D6000BE051092BF051092C0051092C105809368
:101D7000B6059093B705A093B805B093B90508CC04
:101D800081E08CAFA6CC098F1A8F39813B8F4D81B2
:101D90004C8FB8CC20E030E040E05FE3C501B401F7
:101DA0000E94B4379B01AC01632D722D27968FAD35
:101DB000279726969FAD26970E945C34A70196012F
:101DC0000E94B4379B01AC01698D7A8D8B8D9C8DFF
:101DD0000E945C348B0189839D83A5019401632D4E
:101DE000722D27968FAD279726969FAD26970E9436
:101DF0005C347AC05A962D913D914D915C915D97DE
:101E0000C701B6010E94B4374B015C0120E030E00D
:101E100040E05FE30E94B437232D322D27964FAD6B
:101E2000279726965FAD26970E945D34A7019601FD
:101E30000E94B4379B01AC01698D7A8D8B8D9C8D8E
:101E40000E945C348B0189839D839B01AC016E8D64
:101E50007F8D88A199A10E9474371816CCF52E8D1C
:101E60003F8D48A159A16FA178A589A59AA50E9487
:101E70005C349B01AC010E945D346B017C012D89B7
:101E80003E894F89588D632D722D27968FAD2797E8
:101E900026969FAD26970E945D349B01AC01C70139
:101EA000B6010E945C356B017C01BCADB9873D88F1
:101EB0002E88EF892796EFAF2797F88D2696FFAFEC
:101EC00026970E8D1F8D28A1298339A13D8380CCB3
:101ED000A5019401632D722D27968FAD2797269625
:101EE0009FAD26970E945D34362E272E27968FAF02
:101EF000279726969FAF26976BCC2D893E894F89D1
:101F0000588DC701B6010E94B4379B01AC01698DA1
:101F10007A8D8B8D9C8D0E945C348B0189839D838F
:101F20002BA53CA54DA55EA50E94523587FF50CC40
:101F30002BA53CA54DA55EA5698D7A8D8B8D9C8DBD
:101F40000E945C342D893E894F89588D0E945C35F2
:101F50006B017C010BA51CA54DA549835EA55D8386
:101F600082E0898735CC5A962D913D914D915C91B7
:101F70005D97C701B6010E94B4374B015C01AC010B
:101F80009B01632D722D27968FAD279726969FADC7
:101F900026970E947437181664F520E030E040E080
:101FA0005FE3C501B4010E94B4379B01AC01632D0E
:101FB000722D27968FAD279726969FAD26970E9464
:101FC0005C34A70196010E94B4379B01AC01698D76
:101FD0007A8D8B8D9C8D0E945C348B0189839D83CF
:101FE0002FA538A949A95AA90E94743718160CF4CC
:101FF000F4CE2FA538A949A95AA9698D7A8D8B8D60
:102000009C8D0E945C349B01AC010E945D346B018D
:102010007C012DAD3EAD4FAD21965FAD2197632D77
:10202000722D27968FAD279726969FAD26970E94F3
:102030005D349B01AC01C701B6010E945C356B01A8
:102040007C013DAC2EACBFAD2796BFAF2797219644
:10205000EFAD21972696EFAF26970FA518A9F9A9FE
:10206000F9832AA92D83B4CB2DA93EA94FA958AD38
:10207000B80189819D810E94743718168CF42EE373
:1020800033EC4EE259E36BA17CA18DA19EA10E948D
:102090005D346BA37CA38DA39EA3A3019201AECB61
:1020A000832D922D2796AFAD27972696BFAD269705
:1020B0008093B2059093B305A093B405B093B50592
:1020C00049854093AD05BCCB20919D0530919E057F
:1020D00040919F055091A005C301B2010E945D345B
:1020E0002B013C0129853A854B855C85C501B401EE
:1020F0000E945C349B01AC01C301B2010E945C35BB
:102100004B015C0120EC31EE44E65EE40E94B43702
:102110000E943B350E94D535603DA7E07A078105D6
:10212000910508F081C046E029893A89429FF00173
:10213000439FF00D1124EF5DFA4F158246E0298987
:102140003A89429FF001439FF00D1124EF5DFA4F51
:102150007383628380912005809345058F5F86306D
:1021600009F4BBC080932005E091C605F091C70536
:10217000C801A981BD81868F978FA0A3B1A3C0920A
:10218000A105D092A205E092A305F092A4052985AD
:102190003A854B855C85C701B6010E945C34A50178
:1021A00094010E94B43760939D0570939E058093BF
:1021B0009F059093A0052091AE053091AF05409109
:1021C000B0055091B105B80189819D810E945235B9
:1021D000811157C920E030E0A901B80189819D81B2
:1021E0000E94743718160CF07BC08091EA0581605C
:1021F0008093EA05CA5BDF4F0FB6F894DEBF0FBECF
:10220000CDBFDF91CF911F910F91FF90EF90DF90A5
:10221000CF90BF90AF909F908F907F906F905F9086
:102220004F903F902F900895603A5FE075078105C9
:102230009105A0F526E0A989BA892A9FF0012B9F74
:10224000F00D1124EF5DFA4F31E0358346E0298926
:102250003A89429FF001439FF00D1124EF5DFA4F40
:102260002581022E04C096958795779567950A94E7
:10227000D2F7AD85BE8502C0AA0FBB1F2A95E2F733
:10228000B183A08361157105B1E08B07910508F456
:1022900055CF8FEF9FEF938382835CCF60344FE104
:1022A00074078105910560F426E0A989BA892A9FFF
:1022B000F0012B9FF00D1124EF5DFA4F32E0C5CFF6
:1022C000A6E049895A89A49FF001A59FF00D112429
:1022D000EF5DFA4FB3E0B583B9CF1092200544CF3C
:1022E0009BA99111EDCA1092C7051092C605A9AD20
:1022F000BAADAB1709F4C5C8ED8DE03109F41D8EF8
:1023000080913C02FAADF81303C02D8D20933C025E
:102310003D8D30933D02A0C81BAEA7C81BB818B8AE
:1023200080916F008D7F80936F0080918100887F06
:10233000816080938100109218028091260690910E
:10234000E6058F3FA1F42091C905211110C09038F6
:1023500081F490E0019778F481E09091380692FF43
:1023600002C091E08927882369F0289A0895943063
:1023700081F780E0F2CFEFE9FFE03197F1F700C09D
:102380000000E8CF28980895CF93DF930E948E1124
:10239000EBE9F5E08BE2DF011D928A95E9F7C9E1EF
:1023A000D2E083E2FE0111928A95E9F71092C70507
:1023B0001092C60510921F051092450581E080938A
:1023C0002005109218020E94F802209117022F8710
:1023D000E6E1F2E09081937E80911502982B908344
:1023E000E4E1F2E080818F71822B8083DF91CF91D5
:1023F00008958091C80584FD1BC080E10E945402AD
:102400002C9843989091E605892F8C7221F4809145
:10241000EA05867069F0943049F48091C90581110C
:1024200003C086E00E9444020C948E1183E0FACF30
:1024300008952F923F924F925F926F927F928F9268
:102440009F92AF92BF92CF92DF92EF92FF920F9343
:102450001F93CF93DF93CDB7DEB7A4970FB6F89451
:10246000DEBF0FBECDBF1091C905112349F181E038
:102470008093E60583E691E00E948204812F0E940A
:102480005D040E94900485EF91E00197E1F5115001
:10249000123088F486EC92E00E94820484EB92E091
:1024A0000E9482040E94E50580E10E944A02809118
:1024B000C80584FFFCCF8FB7F8941092C9058FBF71
:1024C0001091C805112309F488C214FF23C081E0CC
:1024D0008093E705A4960FB6F894DEBF0FBECDBF7C
:1024E000DF91CF911F910F91FF90EF90DF90CF90F0
:1024F000BF90AF909F908F907F906F905F904F9024
:102500003F902F900895EFE9FFE03197F1F700C079
:102510000000BBCF10FFADC08CE0EDECF5E0DE01BC
:10252000599601900D928A95E1F7BE01675E7F4F43
:10253000CE010D960E9498028CE30E944303809185
:10254000E605883009F40FC108F0EAC0813009F4CB
:1025500013C108F403C1823009F411C1843009F4B5
:1025600008C180912706F82FF1709F2E80FF1CC1B3
:102570008091F205882309F417C18EE891E00E944A
:102580008204CE010D960E9444048091270681FFAB
:102590001DC082E891E00E94820490911E05809106
:1025A0003D02981708F44FC1815F891B0E945D04AA
:1025B0008CE20E94430380911202909113029817BB
:1025C00008F443C18058891B0E945D048EE791E0A6
:1025D0000E9482048091E6058C7709F438C16091ED
:1025E000B2057091B3058091B4059091B5050E9434
:1025F00028040E948208082FF090CC0589E791E01A
:102600000E948204FF2019F080E50E94430300230A
:1026100079F000FF03C088E50E94430301FF03C077
:1026200089E50E94430302FF03C08AE50E94430339
:1026300082E50E94430388E40E94430383E50E94ED
:1026400043038091F205882309F405C181508093EA
:10265000F2050091F105002309F416C10150009321
:10266000F1058EE30E9443030E94900481E00E94E2
:102670004A02812F887E09F460C18091E605982F77
:10268000937009F049C18872A9F08091E805807CB7
:1026900089F40E94D40282E08093EA058091E605E5
:1026A000803241F480E217FD0CC08091E80580681B
:1026B0008093E8058091E605811103C091E0909335
:1026C000E80516FF07C085FD05C09091E8059064F8
:1026D0009093E80513FF05C0807E19F480E1809394
:1026E000E60515FF19C186EC92E00E94820482E79C
:1026F00092E00E9482040E94E5058091E80587FD32
:1027000006C19091E605903409F0FEC083FF04C035
:10271000837E82608093E80580E48093E605F7C0BD
:10272000803221F198F4803109F01BCF8091E805C7
:1027300087FD1CC086EB91E00E9482048091E80531
:1027400080FF2EC080E30E9443030BCF8034D1F082
:10275000803809F006CF85E991E002C080EC91E075
:102760000E948204FECE8CEB91E0FACF82EB91E0E6
:10277000F7CF8DEA91E0F4CF87EA91E0F1CF81EADB
:1027800091E0EECF8BE991E00E9482048091E80510
:1027900083FF02C083E3D7CF82FF04C085FFD2CF7F
:1027A00081E3D1CF82E3CFCF40908406509085065D
:1027B00060908606709087066CE6A62E66E0B62EC0
:1027C0009E012F5F3F4F6901CE010D967C0100E015
:1027D000F50161917191819191915F012085318520
:1027E000428553850E945D34F60161937193819314
:1027F00091936F01023041F4A30192010E945D3474
:1028000069877A878B879C87911012C0F60134976D
:102810002081318142815381F70160817181828100
:1028200093810E945C34F701608371838283938378
:102830000F5FF4E0EF0EF11C033051F691109DCEC6
:1028400087E891E09CCE8150B0CE8150BCCE60E054
:1028500070E0CB01CCCE8091E6058C7799F08DE1CC
:102860008093F2058091F105811103C081E080938E
:10287000F10583E791E00E948204CE0101960E9457
:102880004404E7CE89E0ECCF8091E6058C77A9F18E
:1028900083E18093F1058EE691E00E9482048091AD
:1028A000ED050E945D048CE20E9443038091EE05D9
:1028B0000E945D048CE20E9443038091EF050E9418
:1028C0005D042C9B1CC02D9B1CC052E0F52E439B2D
:1028D000C7C100E48AE691E00E948204FF2031F043
:1028E00021E083E5F21283E40E944303002309F40C
:1028F000B8CE86E40E944303B4CE89E0CACFF12C5F
:10290000E6CFFF24F394E3CF903809F005CF809110
:10291000E80580628093E80517FF0CC08091E6050A
:10292000813029F48091E80585608093E80580E88E
:102930008093E60588EE0E944A0211FF28C0812F8D
:10294000887611F58091E605803441F48091E805A0
:1029500085FD04C084FFE2C01092E6058091E60583
:10296000882309F4E1C084FF0FC09091E80590FF2F
:102970000BC0803109F0D8C08091F005882309F49C
:10298000D3C088608093F00582E00E944A0212FF63
:1029900024C09091E8058091E605807D09F4DDC0B2
:1029A0008091E9058111D9C097FDD9C00E94D40258
:1029B00080913D0280933C020E94C1068091EA050D
:1029C00081FF05C09091E80591609093E805897FAB
:1029D0008093EA0584E00E944A029091CA059923F7
:1029E00009F44CC08FB7F8941092CA058FBF40917C
:1029F000ED05842F90FD84E691FD865F92FD8A505F
:102A000093FD8F5F94FD8150893C08F088EC8A30FB
:102A100008F48AE03091EE05232F95FD24E696FD1B
:102A200022E397FD29E1481302C0231739F180936F
:102A3000ED052093EE051092F10570903D02609037
:102A40001E05172D89E9282E96E7392E26E9422EF4
:102A50003EE7532E4EE2842E16119CC0C101D201D6
:102A60008093220190932301A0932401B093250128
:102A70000E94D40270923C020E94C1061091CB05C4
:102A8000112309F443C08FB7F8941092CB058FBF80
:102A90009091EF05892F10FD84E611FD865F12FDF0
:102AA0008A5013FD8F5F14FD8150893C08F088EC3B
:102AB0008A3008F48AE0981761F09091E6058093D7
:102AC000EF059111C1C0809151060E942E03109212
:102AD000F1058091E60515FF09C0803139F4909128
:102AE000F0059111B7C092E09093F005107C71F061
:102AF000882311F0887351F01091500616FFAEC074
:102B00001F7B812F0E947009109350068091E6056B
:102B10008C7F09F4DFCC0E94F909DCCC82FF1ECF48
:102B200088608093E8051ACF1092EA050E94A906F2
:102B3000892B71F08091E80586FD0AC01092E805A6
:102B400088E08093E6050E94F9090E9415031CCFD6
:102B50001092E8051092E60517CF97FF0AC0109271
:102B6000EA050E947C090E94C4110E94B8080E94D4
:102B700014068091E80585FF08C08F7781608093F7
:102B8000E80580E48093E60525CF1092E8051092D1
:102B9000E60520CFA12EB12C189DC0011124825C26
:102BA0009D4F0E943606962EC72ED82E092F9101D2
:102BB000A2010E9474378A9C70018B9CF00C112436
:102BC0001816ACF5C701825C9D4F7C019101A201F2
:102BD000B101C2010E94B437F701668B778B808FF9
:102BE000918F8A9CC0018B9C900D11249C01225CCA
:102BF0003D4F7901F90122A033A044A055A0A201C4
:102C0000910166897789808D918D0E94743718169D
:102C10002CF4F701268A378A408E518E1F5F1031BF
:102C200009F410E0292C3C2C4D2C502E15CF970187
:102C3000225C3D4F7901292D3C2D4D2D502F692DC2
:102C40007C2D8D2D902FC6CF8091EA0588608093D2
:102C5000EA053DCF90FF4ACF946046CF106451CF34
:102C6000F11038CEFECC1F93CF93DF93142F20E0CA
:102C700030E040EA51E40E94B4370E943B350E94A4
:102C8000D535EB012097C9F08091E705811115C07A
:102C900011110DC00E9461162FEF80E792E02150C4
:102CA00080409040E1F700C000002197EBCF0E94E8
:102CB00019128091E80581FFEFCFDF91CF911F912D
:102CC00008951F93CF93DF930E9419128091E80516
:102CD000882309F453C00E94A906009771F58091DA
:102CE000510690915006892BD82FD07311E0C82F30
:102CF000C07C8091E805882309F440C09091E705E5
:102D000091113CC080FF16C09091E605292F207CD0
:102D100009F47BC082FD1AC01092F00580E00E9489
:102D20002E0380E00E9470098091E8058D7F846009
:102D30008093E8050E941912DCCFFC019189907301
:102D4000439902C080E0CFCF80E4CDCF9038E9F442
:102D500086EC92E00E9482048FE292E00E9482045C
:102D60000E94E50580E00E942E0380E00E94700929
:102D70000E948E118091E705882321F0DF91CF9189
:102D80001F9108950E941912F5CF903419F48F7D88
:102D90008093E8058091E80583FFCCCF90915106A0
:102DA000992359F081FD09C08091380681FF22C026
:102DB0008091EA0588608093EA0580915006882317
:102DC00071F08091E80581FD0AC08C2F0E94700986
:102DD00041E060E070E080E89FE30E94331680915C
:102DE000E80581FDA7CF80618093E80582E00E941D
:102DF0005402A0CF8D2F0E942E0341E060E070E0CE
:102E000080E890E40E943316D8CF8091F0058823A3
:102E1000A1F181FF0AC080915106882339F180E039
:102E20000E942E031093F00585CF8C7009F482CF99
:102E300080915106882399F086EC92E00E948204EA
:102E400088E392E00E9482040E94E50580913806A2
:102E500081FF0FC08091EA0588608093EA05809128
:102E6000F00583FF03C082E00E9454021092F00537
:102E700061CF8D2F0E942E03F2CF8091EA0583FF50
:102E800059CF8D2F0E942E038091EA05877F809372
:102E9000EA0550CF0E94B9060E9461168091E705AD
:102EA000811108C00E94A906892BB1F78091E6051F
:102EB000883091F30895CF93DF9391E5899FE001E6
:102EC0001124DD5F40E550E0BE0182EC96E00E94F7
:102ED0002E09892B79F41092C2060E944A1740E508
:102EE00050E062EC76E0CE010E94DE0880E0DF91E7
:102EF000CF91089581E0FBCF0E944A171092F2050E
:102F00000895CF939091E605923039F0C82F0E9432
:102F10004A178C2FCF910C942E03CF9108950F93C5
:102F20001F93CF93C82F8B010E944A172DE0C29F99
:102F3000C00111244CE050E0B8019E5FCF911F9179
:102F40000F910C94DE081F93CF93DF93182FEB01A2
:102F50008DE0189FB00111247E5F4CE050E0CE015F
:102F60000E942E09892B71F48CE0FE0111928A9542
:102F7000E9F7BE01812F0E948F1780E0DF91CF918A
:102F80001F91089581E0FACFEF92FF920F931F9364
:102F9000CF93DF93CDB7DEB72C970FB6F894DEBF93
:102FA0000FBECDBF182F80FF0BC085E5E5EDF1E02A
:102FB000A3EFB5E005900D928A95E1F70E941909FB
:102FC00011FF10C0CE0101967C018CE0F701119237
:102FD0008A95E9F700E0B701802F0E948F170F5FF5
:102FE0000830C9F712FF14C060E080E093E00E944F
:102FF000BE0860E081E093E00E94BE0860E081E5E9
:1030000093E00E94BE0860E082E593E00E94BE0863
:1030100013FF0AC060E08EEA93E00E94BE0860E001
:103020008FEA93E00E94BE082C960FB6F894DEBF9C
:103030000FBECDBFDF91CF911F910F91FF90EF9009
:1030400008952F923F924F925F926F927F928F924C
:103050009F92AF92BF92CF92DF92EF92FF920F9327
:103060001F93CF93DF93CDB7DEB7C254D1090FB60C
:10307000F894DEBF0FBECDBF3B0100911E05202E90
:10308000312C2EE2029FA0011124BA01625C7D4F17
:103090007AAF69AFFB0111922A95E9F7F301208518
:1030A000FB01218B21FFF0C02CE0EDECF5E0DE010F
:1030B000599601900D922A95E1F789AB9AAB23EFCF
:1030C00035E021963FAF2EAF2197BE01635F7F4F62
:1030D0007EAF6DAFCE0149969CAF8BAFE9ADFAAD37
:1030E000F8AFEFAB9E012B5D3F4F3CAB2BAB3EAB44
:1030F0002DAB10E08EE2829D2001839D500C1124A7
:10310000B201625C7D4F2B01CB010C9623969FAFE1
:103110008EAF239790E1490E511CE9A9FAA961915C
:10312000719181919191FAABE9AB2196EEADFFAD32
:10313000219781909190A190B1902196FFAFEEAF31
:103140002197A50194010E94B4370E948137EDAD0B
:10315000FEAD6193719381939193FEAFEDAFEBADB3
:10316000FCADC190D190E190F190FCAFEBAF6C1948
:103170007D098E099F099B01AC0197FF07C022279B
:103180003327A901261B370B480B590BEFA9F8ADC4
:103190002193319341935193F8AFEFAB2396EEAD6A
:1031A000FFAD2397C080D180E280F380C216D306A2
:1031B000E406F50610F469017A012396EEADFFAD41
:1031C0002397C082D182E282F3820E940636A50153
:1031D00094010E945C35EDA9FEA9619371938193DE
:1031E0009193FEABEDAB20E030E0A9010E94523597
:1031F00087FF0BC090E2112321F090E8113009F411
:1032000090E4F2018081892B80831F5F133009F0E5
:1032100084CF80E0CD28CE28CF2809F4CBC0CE01C2
:1032200085960E948D094B015C012EE2229DC00112
:10323000239D900D11249C01225C3D4F7901F901E1
:10324000868E978EA0A2B1A2BE016B5D7F4F8BE0F0
:1032500096E00E942C08F701628F738F848F958F00
:10326000BE016B5D7F4F8FEF95E00E942C08F70148
:1032700066A377A380A791A7118910FF09C062A751
:1032800073A784A795A710C02CE0EAE0F1E00FCF68
:10329000F301208131814281538113FDA5C0F701E3
:1032A00022A733A744A755A780913D02081711F024
:1032B00011FFA0C08EE2829DF001839DF00D1124CC
:1032C000E25CFD4F128A138A148A158A12A213A295
:1032D00014A215A28EE2829D8001839D100D1124FF
:1032E000025C1D4FF801818981FD63C089AD9AADF3
:1032F0000E9436066B017C01809022019090230190
:10330000A0902401B0902501AC019B01C501B4013E
:103310000E94523587FF36C1A5019401C501B40151
:103320000E94B437F801668B778B808F918F8EE285
:10333000829D8001839D100D1124025C1D4FF801B8
:1033400082A093A0A4A0B5A0A50194016689778965
:10335000808D918D0E94743718162CF4F801868A9E
:10336000978AA08EB18EC0922201D0922301E09262
:103370002401F09225018CE0FE01B596A6E1B1E0B2
:1033800001900D928A95E1F78CE0FE013D96AAE04E
:10339000B1E001900D928A95E1F780910901809347
:1033A0001E058F5F803109F480E0809309010E943F
:1033B000C10681E0CE5BDF4F0FB6F894DEBF0FBED3
:1033C000CDBFDF91CF911F910F91FF90EF90DF90D4
:1033D000CF90BF90AF909F908F907F906F905F90B5
:1033E0004F903F902F900895C501B4010E94B437CB
:1033F000F70145CF26E131E03AAB29AB8E010F5FF3
:103400001F4F6BA97CA9645F7F4F7CAF6BAFC12C52
:10341000D12C76010DAB1FABE9A9FAA9819091904F
:10342000A190B190FAABE9ABEBA9FCA94190519006
:1034300061907190FCABEBABA3019201C501B401AB
:103440000E94B4379B01AC01C701B6010E945C34F5
:103450006B017C01A5019401C301B2010E945C349F
:10346000F80161937193819391938F012BAD3CADE2
:103470006BA97CA92617370779F62FEE3FEF4FE7A8
:103480005FE3C701B6010E94743718164CF48EE250
:10349000829DF001839DF00D1124E25CFD4F16CF5B
:1034A0002FEE3FEF4FE75FEBC701B6010E945235A9
:1034B00087FF11C08EE2829DF001839DF00D1124E3
:1034C000E25CFD4F89E996E7A6E9BEE782A393A3F4
:1034D000A4A3B5A3FFCE8DA99FA90E948D096DA9B4
:1034E0007FA98BE096E00E942C084B015C01A701AC
:1034F000960160E070E080E89FE30E945C3420E089
:1035000030E040E05FE30E94B4370E9453386B0123
:103510007C01209128063091290640912A0650917D
:103520002B06C501B4010E94B437A70196010E9481
:10353000B4374B015C01A701960160E070E080E8C0
:103540009FE30E945C349B01AC01C501B4010E9461
:103550005C356B017C0120E030E0A9010E9452350E
:1035600087FF03C0C12CD12C76018EE2829DF00131
:10357000839DF00D1124E25CFD4FC2A2D3A2E4A210
:10358000F5A2A8CEA7019601C701B601C9CEFF9248
:103590000F931F93CF93DF938C01EB01809138063B
:1035A00085FF23C0F090E60580E2F81611F1C8010E
:1035B0000E945D028823C9F081E08093E90588E0DC
:1035C000F8120CC00E9454020E9461168091E70517
:1035D00081110BC08091E6058111F6CF0E94F9118F
:1035E00082E00E9444020E9461168091E6058230CA
:1035F00021F10E9461168091E70581111EC0909112
:103600003D0280910901981303C00E94B906F1CFD1
:10361000BE01C8010E94211881110FC08091380697
:1036200081FF0BC0888584FF08C080E1DF91CF91C6
:103630001F910F91FF900C948117DF91CF911F91F3
:103640000F91FF9008952F923F924F925F926F9249
:103650007F928F929F92AF92BF92CF92DF92EF9222
:10366000FF920F931F93CF93DF93CDB7DEB7CC5468
:10367000D1090FB6F894DEBF0FBECDBFE8E8F6E083
:103680008AE3DF011D928A95E9F78BE0E8E4F6E032
:10369000A9E8B6E001900D928A95E1F78091C20603
:1036A0008432A1F01A8E1BA2312C212C1EA61DA63D
:1036B00010E01B8E1F8EEE24E394F12CAAE0AA2EBC
:1036C000B12CB1E68B2EB3E09B2E4EC181E08093EE
:1036D000890610928A0683E08A8FB1E0BBA3E4CF0B
:1036E0009FEB9D0D9A3110F00C9498288F5F8A8F74
:1036F000BE016A5E7F4FCE014A960E9485018823F3
:1037000011F40C949B284E885F88688C798CC301D7
:10371000B2010E9497380E94D535062F70E090E0E4
:1037200080E00E9406369B01AC01C301B2010E94F9
:103730005C3420E030E048EC52E40E94B4370E9450
:1037400021380E94D535CB01E7E4DE1629F1FDE4EE
:10375000DF1609F465C1EAEBED0DE53108F02CC088
:103760000E2E000CFF0BE954F44E0C94FF38591D3B
:10377000DC1BDC1B861D911D9C1DA71DDC1BAB1DCE
:10378000DC1BB91DDC1BC31DCD1DD71DDC1BDC1BC9
:10379000DC1BE71DF41D011E083209F4DDC030F505
:1037A000043160F4013108F098C0043009F474C0A9
:1037B000B0F00A3009F468C084E196C00C3109F415
:1037C00063C040F40631C0F725E1201B20938B062F
:1037D00026E087C00E3109F457C0063269F74F8DD5
:1037E00041110C949E28A2E0AF8F28C00D3309F43C
:1037F000AEC0E0F4053309F44FC088F40B3211F089
:103800000133D1F6BF8DB1110C949E28013309F01C
:1038100095C010928E06E3E0EF8F28E04FC00C3386
:1038200058F6065300938F0629E05BC00C3508F567
:103830000A3508F073C0003509F0BECF0093890641
:1038400021E0063209F04DC08431910551F08E31EE
:10385000910539F08832910521F08233910509F004
:10386000ABCFB5010E94C93866576093890621E045
:1038700025C00C3549F00F3508F09ECF2EE5201BF2
:1038800020938A0625E02DC0009731F42F8D211159
:103890000C949E2831E03F8F00938806202F2D7FC7
:1038A0002C3119F020E00C35E1F4009719F00A975B
:1038B00009F082CF600F6093880620E0C70102C044
:1038C000880F991F2A95E2F72DA53EA528233923B5
:1038D000232B09F443C085E107C0015100938D06F5
:1038E00022E0892B59F387E1C45BDF4F0FB6F894D0
:1038F000DEBF0FBECDBFDF91CF911F910F91FF9023
:10390000EF90DF90CF90BF90AF909F908F907F907F
:103910006F905F904F903F902F900895892B29F4DE
:103920000A5500938C0623E0C9CF6A30710509F06F
:1039300043CF0A3509F440CF24E0C0CF0A9709F0FD
:103940003BCFF1E0F0938E0623E02F8F66CF892BDB
:1039500009F032CF2AE0B2CF27E0C3CFADA5BEA594
:10396000A82BB92BBEA7ADA78A8DE82FF0E0EE53A8
:10397000F94FD080D110B4CEBB8DBB2329F0EF8D91
:10398000E11102C0F2E0FF8F25FE0FC08091A50675
:103990009091A606A091A706B091A80681389649F5
:1039A000A849B10514F00C94AA283BA1332309F4CB
:1039B00035C120FE45C180918B068130B1F423E3EF
:1039C00033E34BEC51E4609194067091950680913D
:1039D0009606909197060E94B43760939406709370
:1039E0009506809396069093970630FC10C08091C0
:1039F000530690915406A0915506B09156068093B7
:103A0000B1069093B206A093B306B093B40680912A
:103A10008806843009F02FC126FC2BC18CE164CFCD
:103A2000892B09F060CF063050F4033098F0043051
:103A3000D9F080E10530C9F41092920618C0083020
:103A400008F4BACE0A3048F10E3109F0B5CE009331
:103A5000900604C0002321F00130C9F78BE008C0B4
:103A6000B3E0B0939006FACF80E2809392068CE0A8
:103A7000F70102C0EE0FFF1F8A95E2F7CF012DA5D7
:103A80003EA52E233923232B09F025CF2DA53EA5B6
:103A90002E2B392B3EA72DA767CF093039F0809107
:103AA00091068064809391068DE0E2CF109291069A
:103AB000FBCF4092940650929506609296067092C3
:103AC000970680E06701082E02C0CC0CDD1C0A942A
:103AD000E2F7960122213321232B11F00C94A42824
:103AE000D40102C0B595A7958A95E2F7A0FF0BC057
:103AF00020E030E0A901C301B2010E94523587FFE6
:103B000002C00C94A7282C283D282ECF409298065E
:103B10005092990660929A0670929B06116081E01D
:103B2000D1CF40929C0650929D0660929E06709264
:103B30009F06126082E0C6CF4092A0065092A10676
:103B40006092A2067092A306146083E0BBCF00933C
:103B5000A40684E0B7CFC301B2010E94CE356093C2
:103B6000A5067093A6068093A7069093A80685E005
:103B7000A9CF4092A9065092AA066092AB06709215
:103B8000AC0686E09FCF4092AD065092AE066092A2
:103B9000AF067092B00687E095CF4092B106509282
:103BA000B2066092B3067092B40688E08BCF20E034
:103BB00030E04FE753E4C301B2010E947437181696
:103BC00014F40C94A1280093B50689E07BCF4092B1
:103BD000B6065092B7066092B8067092B9063B8D51
:103BE00031603B8F8AE06ECF4092BA065092BB069E
:103BF0006092BC067092BD064B8D42604B8F8BE08D
:103C000061CF4092BE065092BF066092C00670928D
:103C1000C1068B8D84608B8F8CE054CF80918A0697
:103C2000813081F44F8D423009F0DFCE80918906DA
:103C3000803509F4DACE882309F4D7CE20FCD5CE1E
:103C400086E152CE809149068111CFCE20FCB3CEC1
:103C50008091570690915806A0915906B0915A0646
:103C60008093940690939506A0939606B09397063A
:103C7000BCCEE89426F880918D06882359F08130D7
:103C800009F4BBC022961FAE2297A2E0ABAFB1E011
:103C9000B9AF07C082E022968FAF229791E09BAF29
:103CA00019AE80918B06813071F5E8E8CE2EE6E002
:103CB000DE2EF12CE12C2B8DA22EB12CC5010E2C69
:103CC00002C0959587950A94E2F780FF12C023E31E
:103CD00033E34BEC51E4D6019E966D917D918D912D
:103CE0009C91D1970E94B437F60166A777A780AB65
:103CF00091ABFFEFEF1AFF0A24E0C20ED11C33E0B4
:103D0000E316F104D9F64F8D433049F480918E06C5
:103D1000813029F48B8D843011F00C94AD288CE027
:103D2000ECE6F6E0DE01119601900D928A95E1F73E
:103D3000ADA5BEA5B1FD69C0009188060A3009F4A1
:103D400078C00C3509F419C19F8D933009F43FC038
:103D5000AB8DAA23E1F1B0918C06BFA380918406BC
:103D600090918506A0918606B091870689A79AA7AB
:103D7000ABA7BCA798E4A92E96E0B92E28E8C22EDE
:103D800026E0D22EF12CE12C9B8D892E912CC401A2
:103D90000E2C02C0959587950A94E2F780FD5DC1CF
:103DA000F501808D918DA28DB38DF60186A797A721
:103DB000A0ABB1ABFFEFEF1AFF0A24E0A20EB11CDB
:103DC00034E0C30ED11C43E0E416F10401F70E31D8
:103DD00009F494C1053309F4B8C168E976E086E0D6
:103DE0000C3109F02DC10E94A317882301F18B8D9E
:103DF000811188C119A61F8EA9C0E1E02296EFAFFC
:103E000022971BAEF2E0F9AF4CCF80918F0687303E
:103E100010F08DE169CD90914E06891709F48CCF91
:103E2000BE016F5F7F4F0E94A317811185CF87E08E
:103E30005BCDBB8DB11102C08AE156CDC101807549
:103E40009927892B09F4EACD6091A9067091AA06F9
:103E50008091AB069091AC060E9497380E94D535B0
:103E60006730B8F68091A406843129F0823009F0D9
:103E7000A3CC27FCA1CC662309F474C0615069A7C8
